:020000040000FA
:0400000025EF00F0F8
:0200080034D0F2
:0800180082D0036A026EFF0EA4
:100020000226032200D0D8A01200030E016EE70EB4
:1000300002D8F5D7016AFE0F006EE86A015AD8A00F
:1000400012000000000600D0F8D7F86A4F0EAF6E1D
:10005000240EAC6E900EAB6E0001C69A7F0E926EAF
:10006000E00E936EC60E946E070EB46E0F0EC16E48
:10007000A1D09EAA1BD0060EAB1412E1E1CF26F050
:10008000E2CF27F0282A1EEE80F02850E126000E4D
:10009000E222AECFE7FF26C0E1FF27C0E2FF11005A
:1000A000AE50AE50AB98AB8811000AD0F2A408D085
:1000B000F2940A4A0B2A817A096AD6CF08F0110015
:1000C00011002850295C14E0292AE9CF00F0EACF7A
:1000D00001F00EEE80F02950E926000EEA22EF50E2
:1000E000006E00C0E9FF01C0EAFFD880120004D012
:1000F000E868006ED8A012001200286A296A9D8A5A
:100100009F8AF28EF28C12009D9A0EEE80F0000E05
:10011000EE6AE82EFDD7286A296A9D8A1200F29EAF
:10012000D8CF5AFEE8CF5BFEE0CF5CFEE9CF5DFEA4
:10013000EACF5EFEE1CF5FFEE2CF60FED9CF61FE87
:10014000DACF62FEF6CF63FEF7CF64FEF5CF65FE31
:10015000F3CF66FEF4CF67FEA6CF68FEF28E0001F5
:10016000A192D40EB26EB30EB36EF29E5ACED8FFE9
:100170005BCEE8FF5CCEE0FF5DCEE9FF5ECEEAFF3E
:100180005FCEE1FF60CEE2FF61CED9FF62CEDAFF43
:1001900063CEF6FF64CEF7FF65CEF5FF66CEF3FFC4
:1001A00067CEF4FF68CEA6FFF28E10009EA8FED7A1
:1001B000AD6E120094908B9093988A9893968A963D
:1001C00093948A9493928A9293908A90949A8B9A19
:1001D00094988B9894968B96939A8A9A94908B8005
:1001E000216A94908B90939A8A8A320E16DF939AA2
:1001F0008A9A1F6A256A81DF87DFCD6AF294F28AC4
:10020000870ED56EB16AA192A082B26AB36AD08E0F
:10021000A292B10EB16E55DF0C6EB10E0C5C05E30F
:10022000FE0E0C5C01E20E6A06D10CAE19D00E6A0D
:10023000800E0C5C05E10CC00EF00F6810680FD04A
:10024000900E0C5C05E10CC00EF01168126807D02E
:10025000B00E0C5C04E10CC00EF015681668EBD013
:100260000E5202E1E8D0E7D0800E0E5CD8A449D04F
:100270000F2803E10CC00FF042D00CC010F0240E88
:100280000F5C05E193988A9825901F9037D0250E32
:100290000F5C05E193968A9625921F922FD0260E29
:1002A0000F5C05E193948A9425941F9427D0270E20
:1002B0000F5C05E193928A9225961F961FD0280E17
:1002C0000F5C05E193908A9025981F9817D0290E0E
:1002D0000F5C05E1949A8B9A259A1F9A0FD02A0EEB
:1002E0000F5C05E194988B98259C1F9C07D02B0EE2
:1002F0000F5C04E194968B96259E1F9E0F689BD001
:100300009AD0900E0E5CD8A47DD0112803E10CC0C9
:1003100011F076D00CC012F01252D8A441D0240EA5
:10032000115C05E193988A9825901F9037D0250E8F
:10033000115C05E193968A9625921F922FD0260E86
:10034000115C05E193948A9425941F9427D0270E7D
:10035000115C05E193928A9225961F961FD0280E74
:10036000115C05E193908A9025981F9817D0290E6B
:10037000115C05E1949A8B9A259A1F9A0FD02A0E48
:10038000115C05E194988B98259C1F9C07D02B0E3F
:10039000115C04E194968B96259E1F9E11684BD0AC
:1003A000240E115C03E193988A8829D0250E115CF4
:1003B00003E193968A8623D0260E115C03E1939481
:1003C0008A841DD0270E115C03E193928A8217D094
:1003D000280E115C03E193908A8011D0290E115CE4
:1003E00003E1949A8B8A0BD02A0E115C03E1949856
:1003F0008B8805D02B0E115C02E194968B861168D8
:100400001AD019D0A00E0E5C0AE1132803E10CC02B
:1004100013F003D00CC014F0FAD80DD00CD0B00EED
:100420000E5C09E1152803E10CC015F003D00CC0E7
:1004300016F0F5D800D01F52D8B4E8D01FA01BD0BA
:100440004AC01DF04BC01EF05AC01BF05BC01CF030
:10045000D6CF08F0D7CF09F01B50085C1C500958C4
:100460001D500A581E500B580B501E18D8B0800A49
:10047000D8B8B1EC04F01FA21BD04CC01DF04DC089
:100480001EF05CC01BF05DC01CF0D6CF08F0D7CFCB
:1004900009F01B50085C1C5009581D500A581E508A
:1004A0000B580B501E18D8B0800AD8B8D0EC04F006
:1004B0001FA41BD04EC01DF04FC01EF05EC01BF02D
:1004C0005FC01CF0D6CF08F0D7CF09F01B50085CF6
:1004D0001C5009581D500A581E500B580B501E181E
:1004E000D8B0800AD8B8EFEC04F01FA61BD050C0DB
:1004F0001DF051C01EF060C01BF061C01CF0D6CFD3
:1005000008F0D7CF09F01B50085C1C5009581D504B
:100510000A581E500B580B501E18D8B0800AD8B875
:100520000EEC05F01FA81BD052C01DF053C01EF0EA
:1005300062C01BF063C01CF0D6CF08F0D7CF09F023
:100540001B50085C1C5009581D500A581E500B586F
:100550000B501E18D8B0800AD8B82DEC05F01FAA91
:100560001BD054C01DF055C01EF064C01BF065C008
:100570001CF0D6CF08F0D7CF09F01B50085C1C50F8
:1005800009581D500A581E500B580B501E18D8B051
:10059000800AD8B84CEC05F01FAC1BD056C01DF03B
:1005A00057C01EF066C01BF067C01CF0D6CF08F025
:1005B000D7CF09F01B50085C1C5009581D500A5831
:1005C0001E500B580B501E18D8B0800AD8B86BECD0
:1005D00005F01FAE1BD058C01DF059C01EF068C0FA
:1005E0001BF069C01CF0D6CF08F0D7CF09F01B5024
:1005F000085C1C5009581D500A581E500B580B50CF
:100600001E18D8B0800AD8B88AEC05F004D6136852
:100610001200176812001968120018681200240EE0
:10062000155C0CE12D6A2C6A16C02BF02A6A050EA7
:10063000D8902B362C36E82EFBD774D1250E155CBE
:100640000CE1316A306A16C02FF02E6A050ED89080
:100650002F363036E82EFBD765D1260E155C0CE11F
:10066000356A346A16C033F0326A050ED8903336D4
:100670003436E82EFBD756D1270E155C0CE1396ACB
:10068000386A16C037F0366A050ED89037363836D5
:10069000E82EFBD747D1280E155C0CE13D6A3C6A79
:1006A00016C03BF03A6A050ED8903B363C36E82E31
:1006B000FBD738D1290E155C0CE1416A406A16C09F
:1006C0003FF03E6A050ED8903F364036E82EFBD705
:1006D00029D12A0E155C0CE1456A446A16C043F024
:1006E000426A050ED89043364436E82EFBD71AD11D
:1006F0002B0E155C0CE1496A486A16C047F0466A41
:10070000050ED89047364836E82EFBD70BD1440E5D
:10071000155C13E1066A076A16C005F0046AD890F2
:10072000053204320532043204502A2605502B22A9
:1007300006502C2207502D22F5D0450E155C13E1F2
:10074000066A076A16C005F0046AD89005320432BA
:100750000532043204502E2605502F220650302236
:1007600007503122DFD0460E155C13E1066A076A96
:1007700016C005F0046AD8900532043205320432FE
:1007800004503226055033220650342207503522B9
:10079000C9D0470E155C13E1066A076A16C005F05A
:1007A000046AD890053204320532043204503626E9
:1007B000055037220650382207503922B3D0480E50
:1007C000155C13E1066A076A16C005F0046AD89042
:1007D000053204320532043204503A2605503B22D9
:1007E00006503C2207503D229DD0490E155C13E176
:1007F000066A076A16C005F0046AD890053204320A
:100800000532043204503E2605503F220650402255
:100810000750412287D04A0E155C13E1066A076A29
:1008200016C005F0046AD89005320432053204324D
:1008300004504226055043220650442207504522C8
:1008400071D04B0E155C13E1066A076A16C005F0FD
:10085000046AD89005320432053204320450462628
:100860000550472206504822075049225BD0410ECE
:10087000155CD8A449D02DBE07D02A502B102C10BF
:100880002D1002E01F80258031BE07D02E502F1082
:100890003010311002E01F82258235BE07D0325061
:1008A00033103410351002E01F84258439BE07D080
:1008B000365037103810391002E01F8625863DBEAD
:1008C00007D03A503B103C103D1002E01F882588AD
:1008D00041BE07D03E503F104010411002E01F8A39
:1008E000258A45BE07D0425043104410451002E00F
:1008F0001F8C258C49BE07D0465047104810491020
:1009000002E01F8E258E0ED0420E155C07E11652B6
:1009100003E1219017D801D0218004D07B0E155C13
:10092000D8B402D8156812001F6A206A8A988A967D
:100930008A948A928A908B9A8B988B96939A8A9AA9
:10094000256A12001F6A206A8A988A968A948A9277
:100950008A908B9A8B988B96939A8A9A256A216AA9
:10096000120025B003D01F908A9819D0D6CF08F076
:10097000D7CF09F02A5008241B6E2B5009201C6E7B
:100980002C500A201D6E2D500B201E6E1DC04AF0EB
:100990001EC04BF01BC05AF01CC05BF081781200E7
:1009A00025B203D01F928A9619D0D6CF08F0D7CFA0
:1009B00009F02E5008241B6E2F5009201C6E305059
:1009C0000A201D6E31500B201E6E1DC04CF01EC043
:1009D0004DF01BC05CF01CC05DF08176120025B4A8
:1009E00003D01F948A9419D0D6CF08F0D7CF09F03E
:1009F000325008241B6E335009201C6E34500A20DC
:100A00001D6E35500B201E6E1DC04EF01EC04FF0E7
:100A10001BC05EF01CC05FF08174120025B603D0CD
:100A20001F968A9219D0D6CF08F0D7CF09F036504A
:100A300008241B6E375009201C6E38500A201D6E8A
:100A400039500B201E6E1DC050F01EC051F01BC04F
:100A500060F01CC061F08172120025B803D01F98AD
:100A60008A9019D0D6CF08F0D7CF09F03A50082491
:100A70001B6E3B5009201C6E3C500A201D6E3D50E1
:100A80000B201E6E1DC052F01EC053F01BC062F042
:100A90001CC063F08170120025BA03D01F9A8B9A94
:100AA00019D0D6CF08F0D7CF09F03E5008241B6EDE
:100AB0003F5009201C6E40500A201D6E41500B20F3
:100AC0001E6E1DC054F01EC055F01BC064F01CC04B
:100AD00065F0827A120025BC03D01F9C8B9819D038
:100AE000D6CF08F0D7CF09F0425008241B6E4350F0
:100AF00009201C6E44500A201D6E45500B201E6EAE
:100B00001DC056F01EC057F01BC066F01CC067F039
:100B10008278120025BE03D01F9E8B9619D0D6CFA7
:100B200008F0D7CF09F0465008241B6E4750092023
:100B30001C6E48500A201D6E49500B201E6E1DC0B1
:100B400058F01EC059F01BC068F01CC069F08276D6
:040B50001200FFD7B9
:020000040030CA
:0300010006170ED1
:020005008580F4
:060008000FC00FE00F40E5
:00000001FF
